:100000000C94F1010C9403020C9403020C9403026F
:100010000C9403020C9403020C9403020C9403024C
:100020000C9403020C9403020C9403020C9403023C
:100030000C94B4020C9403020C9403020C94481028
:100040000C9403020C9403020C9403020C9403021C
:100050000C9403020C9403020C9403020C9403020C
:100060000C9403020C9403020C9403020C940302FC
:100070000C9403020C9403020C9494100C9403024D
:100080000C94D0100C9403020C94030286098F097F
:10009000A209A709B109B609C109C812D312E01211
:1000A000F5126213621362136213621362130F1369
:1000B0001C132E134413205354533D005254552007
:1000C0005461736B20657863657074696F6E002589
:1000D000332E3245004E614E0020504F52002045D5
:1000E0005854520020424F52002057445200204A98
:1000F000545200204D435553523D00204B53573628
:100100003830302E3031005044626F7820417070AA
:100110004D61696E00205469636B3D002052584365
:100120003D004D4F42205461736B20004D4F4220E3
:100130004465636F646553656E6420756E73757096
:10014000706F7274656420464E433D004D4F4220EF
:100150004465636F64652057726974653442206535
:1001600072726F720020526567436F756E744F4BE9
:100170003D004D4F42204465636F646553656E6476
:1001800020577269746520464E433432006D6F62A9
:100190005F56616C7565204465636F6465205772B6
:1001A0006974653242206572726F72002052656711
:1001B000436F756E744F4B3D0020526567436F75FA
:1001C0006E743D004D4F42204465636F6465536516
:1001D0006E64206572726F72004D4F422053656EDF
:1001E00064457863657074696F6E2064756D703AEC
:1001F000004D4F422053656E6445786365707469A5
:100200006F6E202D204572726F72436F64653D00E2
:1002100020446174613A0020446174614C656E3D14
:10022000002052656769737465723D004D4F42202E
:1002300052656757726974653432002064756D7059
:100240003A0020446174614C656E3D002052656740
:1002500069737465723D004D4F4220526567577255
:10026000697465313020756E6B6E6F776E00205249
:10027000656769737465723D004D4F422052656732
:1002800052656164303320756E6B6E6F776E002C33
:1002900001000058020000B004000060090000C026
:1002A00012000080250000004B00000096000000B6
:1002B000E1000000C2010000840300000807000004
:1002C000100E0020413D0043464720496E697420CE
:1002D00044656661756C74696E6720436F6E66690C
:1002E000670000000000FFFFFFFFFFFFFFFFFFFFB1
:1002F000FFFFFFFFFFFF0000000000000000000004
:1003000000000000000000000000000000000000ED
:1003100000000000000000000000000000000000DD
:1003200000000000000000000000000000000000CD
:1003300000000000000000000000010000001000AC
:10034000000000010000001000000000010000009B
:100350001000000000010001000000010000000189
:100360000000000100000001000000010000000189
:100370000000000100000002000000020000000276
:100380000000000200000002000000020000000265
:1003900000000002000000000000800000001000CB
:1003A000000020000000400000006000000080000D
:1003B0000000A0000000C0000000E0000000FF00FE
:1003C0000000FFFFFFFF78000000030000000500B1
:1003D0000000040000000000000000000000000019
:1003E000000011241FBECFEFD0E1DEBFCDBF22E061
:1003F000A0E0B1E001C01D92A537B207E1F70E946D
:100400009A140C947E1A0C940000CF93DF934AEA5E
:1004100068E00E940E10C0E0D1E081E089870E9470
:100420006D106A877B878C879D87DF91CF910895B8
:100430000F931F9380E091E00E94A404882309F4A5
:1004400052C080910001882319F0813051F032C0F0
:100450001092090161E080E091E01F910F910C94EE
:100460009004809109018823F9F00E946D10009199
:100470000A0110910B0120910C0130910D01DC015A
:10048000CB01801B910BA20BB30B813D9740A105C3
:10049000B10550F0F89498E088E10FB6F894A8956B
:1004A00081BD0FBE91BDFFCF28EE33E040E050E0AC
:1004B00061E013C08CEB90E00E94010586EB90E0B8
:1004C0000E940105809100010E94F9050E94FB0431
:1004D00020ED37E040E050E060E080E091E01F91E7
:1004E0000F910C9475041F910F91089560E080E0C6
:1004F00091E00C94900480931201482F50E060E04A
:1005000070E08DE20C942C14809112010895809378
:100510001301482F50E060E070E08EE20C942C1440
:1005200080911301089580931401482F50E060E0FA
:1005300070E08FE20C942C1480911401089588309F
:1005400060F4E82FF0E0EE5EFE4F6383462F50E04C
:1005500060E070E0805D0C942C140895E82FF0E0CA
:10056000EE5EFE4F838108951F920F920FB60F9299
:1005700011240BB60F922F933F934F935F936F937A
:100580007F938F939F93EF93FF9380E090E061E0E0
:1005900070E0FC01EE5EFE4F338520911401230FC5
:1005A000238733852381231760F430916200AB01E8
:1005B000082E01C0440F0A94EAF7242F2095232324
:1005C00009C0409162009B01082E01C0220F0A94CD
:1005D000EAF7242B20936200019688309105C9F632
:1005E000FF91EF919F918F917F916F915F914F91CB
:1005F0003F912F910F900BBE0F900FBE0F901F9049
:1006000018950895CF93DF93109262008FEF809337
:1006100061008DE20E941E14609312018EE20E941E
:100620001E14613818F46093130103C080E88093AE
:1006300013018FE20E941E14613118F460931401BB
:1006400003C080E18093140180911401811103C0E3
:1006500081E080931401C0E0D0E08C2F805D0E9487
:100660001E14FE01EE5EFE4F63832196C830D10555
:10067000A1F71FBC8AE08EBD1DBC1CBC809113017C
:1006800090E09BBD8ABD87B7806187BFDF91CF9126
:100690000895883048F49CE1899FF0011124EB5DB6
:1006A000FE4F62870C94E91108952CE1829FC001EE
:1006B0001124FC01EB5DFE4F82850895883070F4B3
:1006C0009CE1899FF0011124EB5DFE4F6387462F6B
:1006D00050E060E070E08B5F0C942C1408952CE1E6
:1006E000829FC0011124FC01EB5DFE4F83850895BC
:1006F000883088F49CE1899FF0011124EB5DFE4F66
:10070000408F518F628F738F4487558766877787B5
:100710008B5E0C942C1408952CE1829FC00111244F
:10072000FC01EB5DFE4F6485758586859785089590
:10073000883068F49CE1899FF0011124EB5DFE4F45
:10074000408B518B628B738B835E0C942C140895B9
:100750002CE1829FC0011124FC01EB5DFE4F6089FA
:100760007189828993890895883068F49CE1899F12
:10077000F0011124EB5DFE4F448B558B668B778B1C
:100780008B5D0C942C1408952CE1829FC0011124E0
:10079000FC01EB5DFE4F6489758986899789089510
:1007A000CF93DF93EC010E94A404882309F457C07F
:1007B0008881813059F118F0823099F150C08B85D1
:1007C0008823F1F0833050F4823051F4888D998D74
:1007D000AA8DBB8D892B8A2B8B2B11F41B8610C005
:1007E00081E08A8761E089850E94E9112889398939
:1007F0004A895B8961E0CE01DF91CF910C94750449
:1008000028EE33E040E050E060E0F5CF1A8660E08B
:1008100089850E94E9112C893D894E895F8962E0B2
:10082000EACF8B858230A9F4888D998DAA8DBB8DF6
:100830000197A109B109888F998FAA8FBB8F892B46
:100840008A2B8B2B31F41A8660E089850E94E9118E
:100850001B8660E0CE01DF91CF910C949004DF9174
:10086000CF910895CF93DF93C5E2D1E0CE010E94EE
:10087000D0036C9682E0C530D807C1F7DF91CF91E5
:1008800008951F93CF93DF93C5E2D1E010E019875D
:1008900085E0810F0E941E146B8785E1810F0E9405
:1008A0001E146C877D878E879F87188E198E1A8EEF
:1008B0001B8E8DE1810F0E941E14688B798B8A8BB1
:1008C0009B8B85E2810F0E941E146C8B7D8B8E8B1F
:1008D0009F8B60E0CE010E9490041F5F6C961830E1
:1008E000B1F6DF91CF911F910895CF92DF92EF92F1
:1008F000FF92CF93DF93EC0169017A0168830E9434
:100900006D1069837A838B839C83CD82DE82EF8234
:10091000F886DF91CF91FF90EF90DF90CF90089510
:100920001F93CF93DF93EC01162F0E946D10698304
:100930007A838B839C8318831D821E821F82188674
:10094000DF91CF911F910895CF92DF92EF92FF92A6
:10095000CF93DF93EC010E946D10C980DA80EB80A9
:10096000FC80DC01CB018C199D09AE09BF0921E097
:10097000CD80DE80EF80F8848C159D05AE05BF0527
:1009800008F420E0822FDF91CF91FF90EF90DF906D
:10099000CF9008959B01280F391F62177307D9F074
:1009A000FB019191BF014927942F92959427092E1D
:1009B000969596959025092E969590259770042EDC
:1009C000452F969507949795502D4927069497950E
:1009D00050254927E2CFCA0108958EE40E942111D3
:1009E00085E50E9421118CE40E9421118CE40C9475
:1009F00021110C9421118DE00E9421118AE00C94A8
:100A00002111CF93DF93EC01892B41F0FE018491FA
:100A1000882341F00E9421112196F8CFDF91CF91D8
:100A20000C94ED04DF91CF910895CF93DF9300975D
:100A300039F0EC018991882339F00E942111FACF15
:100A4000DF91CF910C94ED04DF91CF9108958F70D9
:100A50008A3010F0895C01C0805D0C942111CF9325
:100A6000C82F88E70E9421118C2F82958F700E94D9
:100A700027058C2FCF910C9427050F931F93CF93AD
:100A8000DF938C0188E70E942111CCE0D0E0C801FF
:100A90000C2E02C0969587950A94E2F70E942705CE
:100AA0002497CC3F8FEFD80791F7DF91CF911F911B
:100AB0000F910895CF92DF92EF92FF92CF93DF9341
:100AC0006B017C0188E70E942111CCE1D0E0D701C5
:100AD000C6010C2E04C0B695A795979587950A94E4
:100AE000D2F70E9427052497CC3F8FEFD80779F7DC
:100AF000DF91CF91FF90EF90DF90CF9008954F92CC
:100B00005F926F927F928F929F92AF92BF92CF929D
:100B1000DF92EF92FF920F931F93CF93DF93E82F13
:100B20004A015B019AE0C92ED12CE12CF12CEE2375
:100B300051F0AAE0B0E0A70196010E94EA146B010F
:100B40007C01E150F4CFC0E08AE0482E512C612CAA
:100B5000712CC114D104E104F10429F18C149D0419
:100B6000AE04BF0488F0C501B401A70196010E943C
:100B7000BF148B01D82FC92F80E3820F0E9421114F
:100B80004801AD2EBC2E05C0CC2321F080E30E948D
:100B90002111C1E0C701B601A30192010E94BF1457
:100BA00069017A01D6CFC11113C080E3DF91CF91E3
:100BB0001F910F91FF90EF90DF90CF90BF90AF907B
:100BC0009F908F907F906F905F904F900C94211129
:100BD000DF91CF911F910F91FF90EF90DF90CF9019
:100BE000BF90AF909F908F907F906F905F904F904D
:100BF0000895482F50E060E070E081E00C947F059C
:100C0000AC0160E070E083E00C947F05AB01BC01B7
:100C100088E00C947F050F931F93CF93DF93082FE9
:100C2000C8E0D0E010E8802F812311F081E301C0FB
:100C300080E30E94211116952197A9F7DF91CF91AA
:100C40001F910F9108956F927F928F929F92AF9212
:100C5000BF92CF92DF92EF92FF920F931F93CF93A9
:100C6000DF93CDB7DEB760970FB6F894DEBF0FBE47
:100C7000CDBF6B017C019B01AC010E9471158823E3
:100C800029F085ED90E00E94010589C020E030E068
:100C9000A901C701B6010E94711587FF07C08DE247
:100CA0000E942111F7FAF094F7F8F09420E034E272
:100CB00044E759E4C701B6010E94C9161816C4F4E6
:100CC000FF92EF92DF92CF928FEC90E09F938F9301
:100CD0008E010F5F1F4F1F930F930E944417C8018F
:100CE0000E9415050FB6F894DEBF0FBECDBF57C0EA
:100CF0000CE010E0712C812C84E2982E84E7A82E61
:100D000089E4B82EA5019401C701B6010E947615A9
:100D10000E94E815662E70E080E090E00E941916AF
:100D2000A50194010E94CE169B01AC01C701B6013A
:100D30000E9404156B017C01711002C0662079F0DD
:100D400080E3860D0E94211120E030E040E85FE35F
:100D5000C501B4010E947115882371F010C020E014
:100D600030E040E85FE3C501B4010E9471158111D4
:100D700008C080E30E9421118EE20E942111772495
:100D8000739420E030E040E251E4C501B4010E94D8
:100D900076154B015C010150110909F0B3CF609643
:100DA0000FB6F894DEBF0FBECDBFDF91CF911F917C
:100DB0000F91FF90EF90DF90CF90BF90AF909F90FA
:100DC0008F907F906F9008950F931F93CF938B0117
:100DD000C82FCC2381F0F801808182958F700E940A
:100DE0002705F80181918F010E94270580E20E946A
:100DF0002111C150EECFCF911F910F910895FB01AA
:100E000020813181FC01308321830895FC01DB01C5
:100E10008C9113969C9113979083838311968C9158
:100E2000119712969C91918382830895CF93C4B7B2
:100E30000E94FB040E94FB0487E091E00E940105F0
:100E40008BEF90E00E94010583EF90E00E94010586
:100E50008C2F0E942F05C4FF04C08EEE90E00E94EC
:100E60000105C3FF04C089EE90E00E940105C2FFA6
:100E700004C084EE90E00E940105C1FF04C08EED25
:100E800090E00E940105C0FF04C089ED90E00E943F
:100E90000105CF910C94FB0489E30E941E14862F58
:100EA0006F3F09F488E70895482F50E060E070E054
:100EB00089E30E942C140E944C0780930502089538
:100EC0009091050290930B0290914E0290930C0228
:100ED0009031A1F018F4933031F019C0913419F029
:100EE000923461F014C093E0980F90934C02809379
:100EF0000D02482F50E08EE092E007C096E09093FC
:100F00004C02482F50E08DE092E00E943B17809108
:100F10004C024FEF5FEF6BE072E090E00E94CA047A
:100F2000E0914C02AE2FB0E0AB5FBD4F16968C93B4
:100F300082E08E0F80934C02EF5FF0E0EB5FFD4F9D
:100F4000968389E995E10197F1F700C00E946D1041
:100F5000609306027093070280930802909309023F
:100F60006BE072E080914C020C944A110F931F9336
:100F7000CF93DF93C82F81EF91E00E9401058C2F62
:100F80000E94F9050E94FB0405E012E080914B02EB
:100F9000F801868380914E0280688783C087CCE405
:100FA000D2E083E088834FEF5FEF6BE072E083E095
:100FB00090E00E94CA04E881AE2FB0E0AB5FBD4F65
:100FC00016968C9382E08E0F8883EF5FF0E0EB5FE4
:100FD000FD4F968389E995E10197F1F700C00E94E2
:100FE0006D10F80161837283838394836BE072E0F8
:100FF00088810E944A1189ED91E00E9401056BE011
:1010000072E088810E94E406DF91CF911F910F91D9
:101010000C94FB04CF92DF92EF92FF920F931F93F9
:10102000CF93DF93CDB7DEB7C058D1090FB6F89490
:10103000DEBF0FBECDBF0E946D1060935302709350
:101040005402809355029093560280914E02803153
:10105000F1F118F4833041F018C1813409F474C0FF
:10106000823409F4ABC011C16091510270915202F7
:10107000CB0101978D37910510F082E062C0AE017F
:101080004F5F5F4F80914F02909150020E94570A2C
:10109000882321F0BE016F5F7F4FECC084EC91E0AC
:1010A0000E94010589EB91E00E94010580915102A7
:1010B000909152020E9400068CEA91E00E94010584
:1010C00080E090E00E9400060E94FB04D6C0609180
:1010D000510270915202CB0101978B37910528F58F
:1010E00040914D02242F30E0CB01880F991F281723
:1010F0003907D9F422E132E080914F0290915002F9
:101100000E94160D482F50E020915102309152025A
:101110004217530709F0B1C090914F02209150023D
:1011200029839A831B828C83A1C08DE891E00E9461
:1011300001050E94FB0480914B02882309F4AFC093
:1011400083E00E94B607ABC0809151029091520299
:101150000197CE9780F7C0904F02D0905002E12CBB
:10116000F12C10E0C7018C0D9D1D40914F02509154
:1011700050022091510230915202240F351F8217E4
:10118000930778F461E070E06C0F7D1F610F711DB3
:101190000E94970F180F882321F08FEFE81AF80AA2
:1011A000E1CF8091510290915202E816F90609F0C0
:1011B00064C0BE016F5F7F4F812F5CC08091510280
:1011C000909152029C01215031092E33310508F0D3
:1011D00059C020914D0230E0880F991F880F991F48
:1011E0002817390709F04EC0E0904F02F0905002E6
:1011F00000E010E087E0D82E20914F02309150029D
:101200008091510290915202820F931FE816F906C5
:1012100088F44D2D50E0455F5D4F60914D02C70150
:101220000E94B80F080F111D84E0D80E8FEFE81A46
:10123000F80AE2CF82E791E00E94010585E691E09D
:101240000E940105C8010E9400060E94FB048091D3
:101250005102909152020817190779F480914F02B8
:101260009091500299838A831B830C83BE016F5F28
:101270007F4F84E00E94600712C080914B02882358
:1012800071F0FBCE8CE491E052CF8CE291E00E94B1
:10129000010580914E020E94F9050E94FB04C0588E
:1012A000DF4F0FB6F894DEBF0FBECDBFDF91CF91F9
:1012B0001F910F91FF90EF90DF90CF900895CF9303
:1012C000DF930E940111882309F487C00E946D10EA
:1012D00060930602709307028093080290930902BC
:1012E0000E940611C82F20910A02822F90E0FC0173
:1012F000EB5FFD4FC683422F50E04730510508F0A9
:101300004CC0FA01EA5BFF4F0C94E114C0934B020E
:10131000CC23A9F180910502C8135EC030C0C03152
:1013200041F018F4C33059F404C08FEB8C0F8230B5
:1013300030F487E080934C02C0934E0220C0C093EB
:101340004E024AC010924F02C093500218C08091C2
:101350004F02909150028C2B9093500280934F0239
:101360000EC010925102C093520209C080915102E6
:10137000909152028C2B909352028093510280E004
:1013800025C030914E02303111F0323431F438E062
:101390003C0F30934C02C0934D0230914C0223130A
:1013A000EECF0197D0E0DC2FCC27FC01EB5FFD4FA7
:1013B0002681C22B4FEF5FEF6BE072E00E94CA0400
:1013C000C817D90711F082E001C081E090910A02AC
:1013D0009F5F90930A0201C082E0DF91CF91089550
:1013E0000F931F930E945F09813009F441C020F0E0
:1013F000823009F450C051C080910A02882309F458
:101400004CC00E946D1000910602109107022091BD
:10141000080230910902DC01CB01801B910BA20B69
:10142000B30B4497A105B105C0F182E291E00E949F
:1014300001058CE191E00E94010580910A020E9461
:10144000F90585E191E00E9401050E946D1000916F
:101450000602109107022091080230910902601BD8
:10146000710B820B930B0E9406060E94FB0413C0B3
:1014700063E080E00E94AB120E940A0810920A0208
:101480000E946D1060930602709307028093080219
:101490009093090202C010920A021F910F910895C1
:1014A0000E944C07E5E0F2E08083158208954F9298
:1014B0005F926F927F928F929F92AF92BF92CF92E4
:1014C000DF92EF92FF920F931F93CF93DF9300D0A1
:1014D00000D0CDB7DEB76B017A018C01712C5C01B5
:1014E000A60EB71E74E0672EE1E14E2EF5E05F2EEA
:1014F0000A151B0508F082C2063282E0180709F4BB
:1015000030C208F0C2C00115F2E01F0709F4CFC1D4
:1015100008F079C00832110508F03FC0003211050B
:1015200008F08DC10330110509F458C1D8F4013019
:10153000110509F441C10230110509F051C2F7014A
:10154000E70DF11D108281E0870D8701080F111D45
:101550008BE30E941E14F80160837394739403E07C
:1015600010E0C6CF0D30110509F44BC10E30110546
:1015700009F456C10C30110509F032C2F701E70D2C
:10158000F11D108281E0870DF701E80FF11D5082F7
:10159000739473940DE010E0ABCF0115E1E01E07EA
:1015A00009F461C1A0F4C80180549109089708F0BA
:1015B00017C2F701E70DF11D108281E0870D470189
:1015C000880E911C80EC800F0E94721245C1013080
:1015D00081E0180709F459C10230E1E01E0709F063
:1015E000FFC1F701E70DF11D108281E0870D870132
:1015F000080F111D0E949C02F8018083739473945C
:1016000003E011E075CF0231F2E01F0709F46DC16C
:10161000F0F40430E2E01E0709F485C158F401300B
:1016200082E0180709F44DC10230E2E01E0709F418
:101630005CC1D6C10031F2E01F0709F438C108F0DF
:1016400040C10630E2E01E0709F48BC1C9C1003277
:10165000F2E01F0709F42BC158F40431E2E01E0741
:1016600009F461C10631F2E01F0709F47AC1B8C17B
:10167000023282E0180709F438C108F422C10432AA
:10168000F2E01F0709F44FC1ABC1043582E018072F
:1016900009F449C108F048C00134F2E01F0709F419
:1016A00010C108F50233E2E01E0709F41EC158F428
:1016B000003382E0180709F4FAC00133E2E01E07A4
:1016C00009F4FFC08DC10633F2E01F0709F449C1D8
:1016D000003482E0180709F4EAC00433E2E01E0790
:1016E00009F07EC120C10634F2E01F0709F439C1B8
:1016F00058F40234E2E01E0709F4F7C00434F2E0C3
:101700001F0709F410C16CC1013582E0180709F404
:10171000D8C00235E2E01E0709F4E7C00035F2E068
:101720001F0709F05DC1C3C0003782E0180709F444
:10173000BEC008F50136F2E01F0709F4C2C058F434
:101740000635E2E01E0709F40CC10036F2E01F077F
:1017500009F4ADC045C1043682E0180709F4E3C0BE
:101760000636E2E01E0709F4FCC00236F2E01F076D
:1017700009F036C1BAC0043782E0180709F4D3C0B3
:1017800058F40137F2E01F0709F49BC0023782E0EA
:10179000180709F4AAC024C10115E4E01E0709F4E2
:1017A00000C10130F4E01F0709F40AC1063782E0E6
:1017B000180709F015C1D5C0F701E70DF11D10821A
:1017C00081E0870D8701080F111D0E944C07F80169
:1017D00080837394739402E010E08ACEF701E70DE2
:1017E000F11D108281E0870D8701080F111D8AE32A
:1017F0000E941E14F80160837394739404E010E057
:1018000077CEF701E70DF11D108281E0870DF7011A
:10181000E80FF11D6082739473940EE010E068CEBF
:10182000F701E70DF11D108281E0870DF701E80F48
:10183000F11D4082739473940FE010E059CEF701CC
:10184000E70DF11D108281E0870D4701880E911C84
:1018500080EE800F0E94AE02F40180837394739433
:101860000F5F1F4F45CEF701E70DF11D108281E09C
:10187000870D8701080F111D0E948402F8018083E3
:101880007394739401E011E033CEF701E70DF11D7D
:10189000108281E0870D8701080F111D0E949002C0
:1018A000F80180837394739402E011E021CEC801A3
:1018B000925064E0969587956A95E1F70E945503EA
:1018C0000AC0C8018150924054E0969587955A9578
:1018D000E1F70E946F03F701E70DF11D108291E01F
:1018E000970DF701E90FF11DB8CFF2E0CF16D10443
:1018F00008F486C0C8018250924044E096958795CE
:101900004A95E1F70E948C0369837A838B839C83D9
:10191000BE016F5F7F4FC701870D911D0E940607B3
:1019200084E0780E3BC0E2E0CE16D10408F468C033
:10193000C8018450924034E0969587953A95E1F736
:101940000E94A80369837A838B839C83BE016F5FA7
:101950007F4FC701870D911D0E940607F4E07F0E9F
:101960001DC082E0C816D10408F44AC0C8018650E0
:10197000924024E0969587952A95E1F70E94C4034A
:1019800069837A838B839C83BE016F5F7F4FC7011E
:10199000870D911D0E940607E4E07E0E0E5F1F4F2B
:1019A000A7CDF701E70DF11D108281E0870DF7014A
:1019B000E80FF11D60827394739401E014E098CDF8
:1019C00084B7F701E70DF11D108291E0970DF70143
:1019D000E90FF11D80837394739402E014E088CDC5
:1019E00089E792E00E9401058EE692E00E940105DF
:1019F000C8010E9400060E94FB0402C0872D01C09E
:101A000080E00F900F900F900F90DF91CF911F917A
:101A10000F91FF90EF90DF90CF90BF90AF909F908D
:101A20008F907F906F905F904F9008956F927F920C
:101A30008F929F92AF92BF92CF92DF92EF92FF92DE
:101A40000F931F93CF93DF9300D000D000D0CDB77A
:101A5000DEB78C015B01742E6901F12CE12C842E20
:101A6000912CF71408F04BC2003382E0180709F4F8
:101A70006BC108F0AAC0023082E0180709F48AC1DD
:101A800008F060C032E0632E6F0C08341105A0F539
:101A90000034110508F04BC10330110509F432C1BF
:101AA000E8F40130110509F422C10230110509F0F2
:101AB00005C2F601EF0DF11D418150E060E070E0DC
:101AC0008BE30E942C148BE30E941E14862F0E942D
:101AD0006711E394F62C03E010E0C3CFC8018097B0
:101AE000089708F0EBC1F601EF0DF11D618180EE62
:101AF000800F0E949F0223C1023081E0180709F481
:101B0000ABC1A8F4011581E0180709F49AC10130AE
:101B100081E0180709F0D2C1F601EF0DF11D8181B6
:101B20000E948702E394F62C02E011E09ACF01159F
:101B300082E0180709F408C1013082E0180709F4AF
:101B400015C1BCC1043182E0180709F43EC1E0F4BC
:101B5000003182E0180709F4F7C058F4043082E03D
:101B6000180709F432C1063082E0180709F44EC1A3
:101B7000A5C1013182E0180709F4F8C0023182E002
:101B8000180709F407C19AC1013282E0180709F465
:101B9000EDC058F4063182E0180709F437C100326D
:101BA00082E0180709F4D0C089C1043282E0180726
:101BB00009F40BC1063282E0180709F427C102328A
:101BC00082E0180709F07AC1E5C0043582E0180701
:101BD00009F4FBC008F043C0013482E0180709F49F
:101BE000C5C0E0F4043382E0180709F4EEC058F4ED
:101BF000013382E0180709F4B9C0023382E0180704
:101C000009F4C8C05BC1063382E0180709F4FEC0BE
:101C1000003482E0180709F497C050C1063482E00E
:101C2000180709F4F3C058F4023482E0180709F4E5
:101C3000B1C0043482E0180709F4C7C03FC10135C0
:101C400082E0180709F492C0023582E0180709F40F
:101C5000A1C0003582E0180709F030C175C0003717
:101C600082E0180709F470C008F5013682E0180711
:101C700009F47CC058F4063582E0180709F4C6C0A0
:101C8000003682E0180709F45FC018C1043682E00C
:101C9000180709F49AC0063682E0180709F4B6C09E
:101CA000023682E0180709F009C174C0043782E0E7
:101CB000180709F48AC058F4013782E0180709F4BC
:101CC00055C0023782E0180709F464C0F7C0011557
:101CD00084E0180709F4CBC0013084E0180709F448
:101CE000DAC0063782E0180709F0E8C08FC0F601B5
:101CF000EF0DF11D81810E945407E394F62C02E060
:101D000010E0AFCEF601EF0DF11D418150E060E033
:101D100070E08AE30E942C148AE30E941E14862F2E
:101D20000E945E11E394F62C04E010E09ACEF601D6
:101D3000EF0DF11D618180EC800F0E947C12E39415
:101D40000F5F1F4FF62C8DCEB6016F0D711DCE01AA
:101D500005960E94FF06C801925024E0969587954B
:101D60002A95E1F76D810E94490312C0B6016F0DFB
:101D7000711DCE0105960E94FF06C8018150924058
:101D8000B4E096958795BA95E1F76D810E945E0360
:101D9000E394B0C082E0A816B10408F4B2C0B60162
:101DA0006F0D711DCE0101960E94060749815A816F
:101DB0006B817C81C80182509240A4E09695879502
:101DC000AA95E1F70E9478031AC082E0A816B10430
:101DD00008F497C0B6016F0D711DCE0101960E94E7
:101DE000060749815A816B817C81C80184509240E9
:101DF000F4E096958795FA95E1F70E949803E394AD
:101E0000E3940E5F1F4F84E0F80E2BCE82E0A816FD
:101E1000B10408F476C0B6016F0D711DCE010196B4
:101E20000E94060749815A816B817C81C8018650D6
:101E30009240E4E096958795EA95E1F70E94B40315
:101E4000DECFF601EF0DF11D81810E947B02E3944C
:101E5000F62C01E011E005CEF601EF0DF11D8181B8
:101E60000E949302E394F62C03E011E0FACDF60110
:101E7000EF0DF11D808190E0982F88272181820F3E
:101E8000911D9E838D830E940502E394F394F39445
:101E900001E014E0E6CDF601EF0DF11D808190E048
:101EA000982F88272181820F911D9E838D8384BF67
:101EB000E394F394F39402E014E0D3CD87E592E049
:101EC0000E9401058CE492E00E940105C8010E9475
:101ED000000682E492E00E940105C4010E9400060F
:101EE0008BE392E00E940105B601872D0E94E40673
:101EF0000E94FB040F5F1F4FF394F394B2CD8E2D1D
:101F000001C080E026960FB6F894DEBF0FBECDBFAD
:101F1000DF91CF911F910F91FF90EF90DF90CF90C5
:101F2000BF90AF909F908F907F906F900895CF93C8
:101F3000DF93EB018431910561F020F44397A1F424
:101F400081E00AC08531910531F0469769F484E05B
:101F500003C082E001C083E00E941E14688379837D
:101F60008A839B8384E001C080E0DF91CF91089554
:101F7000FF920F931F93CF93DF93EC01F62E8A010C
:101F80008CE292E00E94010581E292E00E9401054C
:101F9000CE010E94000687E192E00E9401058F2D8C
:101FA00090E00E94000680E192E00E940105B801E5
:101FB00084E00E94E4060E94FB04C431D105B1F024
:101FC00048F4639721F5F801408151816281738162
:101FD00081E019C0C531D10581F06697C1F4F801DF
:101FE000408151816281738184E00DC0F80140819C
:101FF00051816281738182E006C0F8014081518184
:102000006281738183E00E942C1481E001C080E032
:10201000DF91CF911F910F91FF900895FF920F9341
:102020001F93CF93DF93CDB7DEB760970FB6F894C9
:10203000DEBF0FBECDBFF82E062F142F40E150E0BB
:1020400068E170E0CE0101960E942D1AF9820A83A0
:102050001B834FEF5FEFBE016F5F7F4F8EE090E01D
:102060000E94CA04988B8F8740E150E068E170E0DD
:10207000CE0101960E94431A60960FB6F894DEBF17
:102080000FBECDBFDF91CF911F910F91FF900895AB
:102090001F920F920FB60F9211248F939F93AF93BD
:1020A000BF938091750290917602A0917702B091D2
:1020B00078020196A11DB11D80937502909376025E
:1020C000A0937702B0937802BF91AF919F918F91C7
:1020D0000F900FBE0F901F901895F89460917502A5
:1020E00070917602809177029091780278940895A9
:1020F0008CE083BF8BEA81BF82E087BF80E888B92C
:1021000010BC9FE088E10FB6F894A89581BD0FBE82
:1021100091BD78940895A89585B7837E85BF85B7CE
:10212000806285BF889508951F920F920FB60F9217
:1021300011240BB60F922F938F939F93EF93FF93DE
:1021400091E080919B0087FF1FC020919C008C71C3
:10215000C1F7E0910303F0E0E758FD4F2083809141
:1021600003038F5F809303038A3811F410920303F3
:10217000809105038F5F809305038A3811F71092D1
:10218000050390930603DDCFFF91EF919F918F910F
:102190002F910F900BBE0F900FBE0F901F901895B0
:1021A0001F920F920FB60F9211240BB60F928F93BE
:1021B000EF93FF93809193038823B9F08091930369
:1021C000815080939303E0919203F0E0E95FFC4F2C
:1021D000808180939C00809192038F5F8093920313
:1021E0008A3829F41092920302C010929403FF914E
:1021F000EF918F910F900BBE0F900FBE0F901F901D
:102200001895F894809105037894089580910503BA
:102210008823E1F3E0910403F0E0E758FD4F80816B
:10222000909104039F5F909304039A3811F41092E5
:102230000403F894909105039150909305037894CA
:102240000895909193039A38E1F391E09093940369
:10225000F89490919303911104C090919B0095FD87
:1022600015C0E0919103F0E0E95FFC4F808380911D
:1022700091038F5F809391038A3811F41092910338
:10228000809193038F5F8093930302C080939C009F
:10229000789408950F931F93CF93DF93EB018B01F5
:1022A000080F111DC017D10721F089910E9421113B
:1022B000F9CFDF91CF911F910F91089510929B005C
:1022C00088ED80939A0086E080939D0008958E3F6C
:1022D00009F485E00E949F119B01AC0184E0220F6C
:1022E000331F441F551F8A95D1F760E070EC88EAD0
:1022F00090E00E94BF14DA01C9010197A109B10958
:10230000892F9A2FAB2FBB278093980021502093C1
:10231000990008951092030310920403109205038C
:1023200010929403109291031092920310929303CF
:102330008B9A85E00E94671183E00C945E118D30CA
:1023400008F085E094E0899FF0011124E157FD4FEA
:102350006591759185919491089595B3892B85BB6D
:10236000089595B38095982395BB08958330E1F047
:1023700030F4813081F098F485B381700895853010
:10238000E1F0B8F08630F1F0863409F585B3881FA6
:102390008827881F089585B386958170089585B331
:1023A00082FB882780F9089585B383FB882780F90D
:1023B000089585B382958170089585B385FB88273C
:1023C00080F9089585B386FB882780F9089580E019
:1023D0000895CF93DF93C82FD62F0E94B611C33034
:1023E000F9F020F4C13081F048F014C0C53021F17B
:1023F000E8F0C63039F1C63459F12FC0DD2311F0B1
:10240000A8982BC0A89A29C0DD2311F0A99825C04F
:10241000A99A23C0DD2311F0AA981FC0AA9A1DC053
:10242000DD2311F0AB9819C0AB9A17C0D11102C0CF
:10243000AC9813C0AC9A11C0D11102C0AD980DC0B8
:10244000AD9A0BC0D11102C0AE9807C0AE9A05C0BC
:10245000D11102C0AF9801C0AF9ADF91CF9108951A
:10246000CF9315BA8FEF84BBC0E060E08C2F0E9441
:10247000E911CF5FC830C9F7CF910895282F811196
:1024800006C0662311F01A9804C01A9A10C0662379
:1024900071F081E090E002C0880F991F2A95E2F761
:1024A0002091570230915802822B932B0FC081E06C
:1024B00090E002C0880F991F2A95E2F780959095C9
:1024C000209157023091580282239323909358020F
:1024D0008093570208951A9A129A109258021092F5
:1024E00057020895883030F4E82FF0E0E75AFD4FA6
:1024F0008081089580E00895883028F4E82FF0E086
:10250000E75AFD4F6083E9E5F2E080E090E02FEFCD
:1025100061E070E03191332341F0AB01082E01C03E
:10252000440F0A94EAF740952423019688309105D8
:1025300089F72BBB08958FEF8BBB8ABBE9E5F2E0EF
:10254000119282E0E136F807D9F70895809173027D
:10255000909174020895CF93DF93C82FD0E092E159
:10256000899FD0011124AF59BD4F19969C9119979D
:10257000961709F4A7C019966C93462F50E04E3079
:10258000510508F09FC0FA01E35BFF4F0C94E11482
:1025900060E00E943E1222E12C9FC0012D9F900D11
:1025A000112460E00AC061E00E943E1222E12C9FEB
:1025B000C0012D9F900D112461E08F599D4F7EC069
:1025C00022E12C9FC0012D9F900D11248F599D4F0A
:1025D00040E550E060E070E0FC014287538764878B
:1025E00075874FEF5FEFBA0164C022E12C9FC001F5
:1025F0002D9F900D11248F599D4F4FEF5FEFBA0122
:10260000FC01428753876487758740E550E060E0AE
:1026100070E046875787608B718B63E04FC022E183
:102620002C9FC0012D9F900D11248F599D4F48EC78
:1026300050E060E070E00CC022E12C9FC0012D9FB3
:10264000900D11248F599D4F44E650E060E070E0FA
:10265000FC0142875387648775872BC022E12C9F3A
:10266000C0012D9F900D11248F599D4F42E350E0E2
:1026700060E070E0FC01428753876487758748EE0D
:1026800053E060E070E015C022E12C9FC0012D9F57
:10269000900D11248F599D4F42E350E060E070E0AF
:1026A000FC01428753876487758746E553E160E004
:1026B00070E046875787608B718B62E0DF91CF9126
:1026C0000C949004DF91CF91089522E1829FC00184
:1026D0001124FC01EF59FD4F818508951F93CF937D
:1026E000DF93182F82E1189FE0011124CF59DD4FAD
:1026F000CE010E94A404882309F495C0888181300A
:1027000021F130F08230E1F1833009F45EC08BC0FA
:1027100060E0812F0E943E1281E090E002C0880FAD
:10272000991F1A95E2F78095909520917302309148
:10273000740282239323909374028093730228EE91
:1027400033E040E050E060E068C061E0812F0E942B
:102750003E1281E090E002C0880F991F1A95E2F7BF
:102760002091730230917402822B932B9093740208
:102770008093730228EE33E040E050E061E04DC00A
:1027800061E0812F0E943E1281E090E002C0880F3C
:10279000991F1A95E2F72091730230917402822BEF
:1027A000932B90937402809373022A853B854C850A
:1027B0005D852F3F8FEF38074807580721F481E0E8
:1027C000898761E023C063E028C060E0812F0E9418
:1027D0003E1281E090E002C0880F991F1A95E2F73F
:1027E0002091730230917402822B932B9093740288
:1027F000809373022E853F85488959892F3F8FEF3B
:1028000038074807580741F4198660E0CE01DF9188
:10281000CF911F910C94900462E0CE01DF91CF9193
:102820001F910C947504DF91CF911F91089580E062
:102830000C946E1361E080E00C94AB12803440F491
:1028400024E0829FC001112480589F4F0C943D1AB0
:1028500060E070E0CB010895803440F424E0829F72
:10286000C001112480589F4F0C94641A0895CF9290
:10287000DF92EF92FF920F931F93CF93DF9380E746
:1028800091E00E943D1AE2EDF3E00591159125914A
:102890003491601771078207930709F442C087ECEF
:1028A00092E00E94010583EC92E00E94010580E81D
:1028B00090E00E943D050E946D106B017C01C2EE0C
:1028C000D2E000E810E0FE014591559165917491C8
:1028D000C8010E94641A0E946D10DC01CB018C19A2
:1028E0009D09AE09BF09893C9105A105B10540F0DC
:1028F000A8958EE20E94F9040E946D106B017C0184
:1029000024960C5F1F4F83E0C23ED807E1F6DF91AB
:10291000CF911F910F91FF90EF90DF90CF900C948B
:10292000FB04DF91CF911F910F91FF90EF90DF900B
:10293000CF9008950E9478100E9430120E949B123E
:102940000E946B120E948A110E9416070E9437147F
:102950000E9441040E9402030E9476020E94500AD3
:102960000E941A140E9432040E9401030E9418025D
:102970000E94F0090E9417140E948B10F3CFA1E26D
:102980001A2EAA1BBB1BFD010DC0AA1FBB1FEE1FE9
:10299000FF1FA217B307E407F50720F0A21BB30B34
:1029A000E40BF50B661F771F881F991F1A9469F7B0
:1029B00060957095809590959B01AC01BD01CF010C
:1029C0000895EE0FFF1F0024001C0BBE0790F69128
:1029D000E02D09940E94F514A59F900DB49F900DD1
:1029E000A49F800D911D11240895A29FB001B39F53
:1029F000C001A39F700D811D1124911DB29F700D08
:102A0000811D1124911D08955058BB27AA270E94AB
:102A10001C150C948F160E94811638F00E9488169F
:102A200020F039F49F3F19F426F40C947E160EF42E
:102A3000E095E7FB0C947816E92F0E94A01658F356
:102A4000BA17620773078407950720F079F4A6F593
:102A50000C94C2160EF4E0950B2EBA2FA02D0B018C
:102A6000B90190010C01CA01A0011124FF27591BD3
:102A700099F0593F50F4503E68F11A16F040A22FD9
:102A8000232F342F4427585FF3CF4695379527954A
:102A9000A795F0405395C9F77EF41F16BA0B620B49
:102AA000730B840BBAF09150A1F0FF0FBB1F661F90
:102AB000771F881FC2F70EC0BA0F621F731F841FD3
:102AC00048F4879577956795B795F7959E3F08F0F9
:102AD000B0CF9395880F08F09927EE0F97958795BB
:102AE00008950E94541608F481E008950E948A1502
:102AF0000C948F160E94881658F00E94811640F0A0
:102B000029F45F3F29F00C94781651110C94C316E8
:102B10000C947E160E94A01668F39923B1F35523F6
:102B200091F3951B550BBB27AA27621773078407E0
:102B300038F09F5F5F4F220F331F441FAA1FA9F376
:102B400035D00E2E3AF0E0E832D091505040E69564
:102B5000001CCAF72BD0FE2F29D0660F771F881FC5
:102B6000BB1F261737074807AB07B0E809F0BB0BB8
:102B7000802DBF01FF2793585F4F3AF09E3F5105CC
:102B800078F00C9478160C94C3165F3FE4F3983EEB
:102B9000D4F3869577956795B795F7959F5FC9F7B5
:102BA000880F911D9695879597F90895E1E0660F36
:102BB000771F881FBB1F621773078407BA0720F0AF
:102BC000621B730B840BBA0BEE1F88F7E095089518
:102BD0000E94A81688F09F5798F0B92F9927B751EF
:102BE000B0F0E1F0660F771F881F991F1AF0BA95B1
:102BF000C9F714C0B13091F00E94C216B1E0089537
:102C00000C94C216672F782F8827B85F39F0B93F28
:102C1000CCF3869577956795B395D9F73EF4909563
:102C20008095709561957F4F8F4F9F4F0895E894E1
:102C300009C097FB3EF490958095709561957F4F04
:102C40008F4F9F4F9923A9F0F92F96E9BB279395B2
:102C5000F695879577956795B795F111F8CFFAF4C2
:102C6000BB0F11F460FF1BC06F5F7F4F8F4F9F4FF3
:102C700016C0882311F096E911C0772321F09EE851
:102C8000872F762F05C0662371F096E8862F70E0B7
:102C900060E02AF09A95660F771F881FDAF7880F91
:102CA0009695879597F90895990F0008550FAA0BE7
:102CB000E0E8FEEF16161706E807F907C0F012164F
:102CC0001306E407F50798F0621B730B840B950B52
:102CD00039F40A2661F0232B242B252B21F40895A7
:102CE0000A2609F4A140A6958FEF811D811D089544
:102CF00097F99F6780E870E060E008959FEF80ECAF
:102D0000089500240A941616170618060906089551
:102D100000240A9412161306140605060895092EB7
:102D20000394000C11F4882352F0BB0F40F4BF2B26
:102D300011F460FF04C06F5F7F4F8F4F9F4F089566
:102D400057FD9058440F551F59F05F3F71F047955C
:102D5000880F97FB991F61F09F3F79F08795089541
:102D6000121613061406551FF2CF4695F1DF08C060
:102D7000161617061806991FF1CF8695710561057D
:102D800008940895E894BB2766277727CB0197F925
:102D900008950E94541608F48FEF08950E94E116DA
:102DA0000C948F160E94811638F00E94881620F02D
:102DB000952311F00C9478160C947E1611240C9423
:102DC000C3160E94A01670F3959FC1F3950F50E0B3
:102DD000551F629FF001729FBB27F00DB11D639FCD
:102DE000AA27F00DB11DAA1F649F6627B00DA11D73
:102DF000661F829F2227B00DA11D621F739FB00D19
:102E0000A11D621F839FA00D611D221F749F332788
:102E1000A00D611D231F849F600D211D822F762F21
:102E20006A2F11249F5750409AF0F1F088234AF0FE
:102E3000EE0FFF1FBB1F661F771F881F915050406A
:102E4000A9F79E3F510580F00C9478160C94C31698
:102E50005F3FE4F3983ED4F3869577956795B795F1
:102E6000F795E7959F5FC1F7FE2B880F911D96950B
:102E7000879597F90895FB01DC0102C001900D923E
:102E800041505040D8F708950F931F93CF93DF938D
:102E9000CDB7DEB72E970FB6F894DEBF0FBECDBF0D
:102EA0000D891E898EE08C831A8309838FEF9FE73B
:102EB0009E838D83AE01475E5F4F6F89788DCE0113
:102EC00001960E947317EF81F885E00FF11F1082C1
:102ED0002E960FB6F894DEBF0FBECDBFDF91CF9117
:102EE0001F910F9108952F923F924F925F926F9290
:102EF0007F928F929F92AF92BF92CF92DF92EF928A
:102F0000FF920F931F93CF93DF93CDB7DEB72B972D
:102F10000FB6F894DEBF0FBECDBF6C017B018A01F6
:102F2000FC0117821682838181FFCCC1CE010196FC
:102F30003C01F6019381F70193FD859193FF819107
:102F40007F01882309F4BAC1853239F493FD859154
:102F500093FF81917F01853229F4B60190E00E94B0
:102F60009319E7CF912C212C312CFFE1F315D8F0E8
:102F70008B3279F038F4803279F08332A1F4232D4A
:102F800020611DC08D3261F0803369F4232D2160F2
:102F900016C0832D8260382EE32DE4603E2E2AC0B9
:102FA000F32DF8601DC037FC2DC020ED280F2A300E
:102FB00040F08E32B9F436FC81C1232D2064322ECC
:102FC00019C036FE06C08AE0989E200D1124922E6C
:102FD00011C0EAE02E9E200D1124222EF32DF06266
:102FE0003F2E08C08C3621F4832D8068382E02C015
:102FF000883641F4F70193FD859193FF81917F011C
:103000008111B3CF982F9F7D9554933028F40C5F96
:103010001F4F9FE399830DC0833631F0833771F0E2
:10302000833509F059C021C0F801808189830E5F82
:103030001F4F88248394912C530113C02801F2E080
:103040004F0E511CF801A080B18036FE03C0692DDF
:1030500070E002C06FEF7FEFC5010E9488194C013C
:103060008201F32DFF773F2E16C0280122E0420E89
:10307000511CF801A080B18036FE03C0692D70E0BC
:1030800002C06FEF7FEFC5010E947D194C01F32D47
:10309000F0683F2E820133FC1BC0822D90E0881621
:1030A0009906B0F4B60180E290E00E9493192A9448
:1030B000F4CFF50137FC859137FE81915F01B601B0
:1030C00090E00E94931921102A9421E0821A91081D
:1030D0008114910471F7E8C0843611F0893641F506
:1030E000F80137FE07C060817181828193810C5F96
:1030F0001F4F08C060817181072E000C880B990B4F
:103100000E5F1F4FF32DFF763F2E97FF09C090955E
:103110008095709561957F4F8F4F9F4FF0683F2E40
:103120002AE030E0A3010E94CF19882E861845C0FE
:10313000853731F4232D2F7EB22E2AE030E025C0D2
:10314000932D997FB92E8F36C1F018F4883579F018
:10315000B5C0803719F0883721F0B0C0E92FE061A1
:10316000BE2EB4FE0DC0FB2DF460BF2E09C034FE90
:103170000AC0292F2660B22E06C028E030E005C024
:1031800020E130E002C020E132E0F801B7FE07C0E4
:1031900060817181828193810C5F1F4F06C06081C5
:1031A000718180E090E00E5F1F4FA3010E94CF1954
:1031B000882E8618FB2DFF773F2E36FE0DC0232D5F
:1031C0002E7FA22E891458F434FE0BC032FC09C0A5
:1031D000832D8E7EA82E05C0B82CA32C03C0B82C3E
:1031E00001C0B92CA4FE0FC0FE01E80DF11D8081C5
:1031F000803321F49A2D997EA92E09C0A2FE06C023
:10320000B394B39404C08A2D867809F0B394A3FCD8
:1032100011C0A0FE06C0B21488F4280C922C9B1892
:103220000EC0B21460F4B60180E290E00E949319DF
:10323000B394F7CFB21418F42B1802C0982C212C99
:10324000A4FE10C0B60180E390E00E949319A2FE94
:1032500017C0A1FC03C088E790E002C088E590E0B9
:10326000B6010CC08A2D867859F0A1FE02C08BE20F
:1032700001C080E2A7FC8DE2B60190E00E949319A4
:10328000891438F4B60180E390E00E9493199A946F
:10329000F7CF8A94F301E80DF11D8081B60190E02B
:1032A0000E9493198110F5CF222009F442CEB60175
:1032B00080E290E00E9493192A94F6CFF60186816D
:1032C000978102C08FEF9FEF2B960FB6F894DEBF69
:1032D0000FBECDBFDF91CF911F910F91FF90EF9067
:1032E000DF90CF90BF90AF909F908F907F906F9026
:1032F0005F904F903F902F900895FC010590615092
:1033000070400110D8F7809590958E0F9F1F0895FB
:10331000FC016150704001900110D8F780959095A4
:103320008E0F9F1F08950F931F93CF93DF93FB0181
:10333000238121FD03C08FEF9FEF2CC022FF16C019
:1033400046815781248135814217530744F4A08177
:10335000B1819D012F5F3F4F318320838C93268164
:1033600037812F5F3F4F3783268314C08B01EC01D9
:10337000FB010084F185E02D0995892BE1F6D80148
:1033800016968D919C911797019617969C938E9304
:103390001697CE01DF91CF911F910F910895FA01F9
:1033A000AA27283051F1203181F1E8946F936E7F84
:1033B0006E5F7F4F8F4F9F4FAF4FB1E03ED0B4E075
:1033C0003CD0670F781F891F9A1FA11D680F791FB6
:1033D0008A1F911DA11D6A0F711D811D911DA11DC7
:1033E00020D009F468943F912AE0269F11243019D7
:1033F000305D3193DEF6CF010895462F4770405D72
:103400004193B3E00FD0C9F7F6CF462F4F70405D20
:103410004A3318F0495D31FD4052419302D0A9F77B
:10342000EACFB4E0A6959795879577956795BA9575
:10343000C9F700976105710508959B01AC010A2E3B
:1034400006945795479537952795BA95C9F7620F12
:10345000731F841F951FA01D0895DC01CB01FC0183
:10346000E199FECF06C0FFBBEEBBE09A31960DB2EC
:103470000D9241505040B8F70895A6E1B0E044E005
:1034800050E00C942F1ADC01A40FB51F415050409E
:1034900048F0CB01840F951F2E910E94541A415081
:1034A0005040D0F70895262FE199FECF9FBB8EBBE9
:1034B000E09A01970DB2021631F02DBB0FB6F894C9
:1034C000E29AE19A0FBE0895242F0E94721A252FC6
:1034D0000E94721A0C946C1A0E94711A272F0C9475
:1034E000721A262FE199FECF9FBB8EBB2DBB0FB664
:1034F000F894E29AE19A0FBE01960895F894FFCFEE
:00000001FF
